:020000020000FC
:1000000001C014C14CEA4DBFBB27DD27FF271124D7
:1000100042E0142AEE245AD26BD231D2DFD144E02E
:1000200048BB40EC45BB4BE742BB40E041BB4427EB
:100030004FBB46E846B940E447B94FE045BF40E40E
:100040004BBF7894B09B07C0023079F0033051F079
:1000500010FC13C0F7CF4FEFB099F4CF4A95E1F7FA
:10006000BDD1F0CF07D404E0EDCFC0E66C2D56D261
:10007000D9D264D24BD304E0E5CF412D4FEF4D7F71
:100080004E7F142214FC55C041E04093B40040E080
:100090009AD04093B9003093BA00132F41E093D027
:1000A0008894441F331F441F331F142B306C10934C
:1000B000BA003093BB0042E097D04093B50043E0D4
:1000C00093D04093B60044E08FD04093B70045E012
:1000D0008BD04093B8008F9A97986CD0979AA79836
:1000E000487711F440EF1DC043FF0AC044FF02C02F
:1000F00040E117C046FF02C040E713C040E011C016
:1001000045FF0AC044FF02C040E30BC046FF02C0E7
:1001100040E507C040E405C044FF02C040E201C022
:1001200040E63091BB003F70342B3093BB0018E0A9
:1001300035C042E04093B400BB9AC3983BD0C39A09
:10014000BB98142FBC9AC49835D0C49ABC984795D4
:1001500037953078132B1093B5004F73142FBD9A39
:10016000C59828D0C59ABD98479537954795379536
:10017000307C132B1093B6004F71142F8F9A9798E1
:1001800019D0979AA79847953795479537954795EA
:100190003795307E132B1093B70014E040E11426FE
:1001A0004DEF4F9340E04F93C2EB62E0610FCF936E
:1001B0006F934DC2000040B34B7736B33470432B7E
:1001C00040954F7708954770406447B9369A3699FD
:1001D000FECF44B135B1403019F4303009F441E07C
:1001E00040503240337008954770406647B9369AA0
:1001F0003699FECF45B140580895639563954D2DCE
:100200004093AF00482D4093AE009394C2EB96D13B
:1002100099246093B1008092B0004091AF00D42E39
:100220004091AE00842E42E0142A0CCF5FB64F936B
:100230003F9343E032E0B09BFECFB19BFECFB19B3A
:1002400005C043E03A95000099F0F9CF32E04A95B5
:100250000000A9F707C06F90AF911F912F91CF9128
:100260006F91522D3F914F915FBE80E48ABF1895E8
:10027000252E86B36F93CF9356E06EE0CEE676B32D
:100280007370A1F07795881F5A95C9F7000076B36F
:10029000737061F07795881F57E0899386B38370F8
:1002A00029F05A9500006A9551F7D9CFC137B8F2B5
:1002B00040916E0030916F0071F43E7F3F1559F40C
:1002C000423711F491E0CBCF403511F493E0C7CF22
:1002D0004E3409F40AC0483211F0463321F491300B
:1002E00001F1933031F190E0BACF2F931F93AF9388
:1002F0006F9230916F00209170003795279522956D
:1003000030FF01C020952F702A3019F02530E9F018
:10031000A2CF0430B9F46CD0EE20B1F492E003E047
:100320009ACF2F931F93AF936F92D7D040D002E014
:1003300092CF2F931F93AF936F92023019F0CDD0CD
:10034000002789CFDCD087CF22C011FE1FC04D2DE2
:100350004093AF00482D4093AE004091B000842EF2
:100360006091B100C2EB46D04091AF00D42E4091D5
:10037000AE00842E4091B300433C11F043EC01C029
:100380004BE44093B30041E0142A65CF64CFFF24CF
:1003900021E018E04F2DE79408F042274795FF1C15
:1003A0001A95C1F7EE242F2D2E7FF22E54CF573001
:1003B00029F05395881F5A95E9F789936C2F6D564C
:1003C000C62ECEE6A1E6BF93BB2749914D936A9511
:1003D000E1F7BF9164E56093600008954AEAF42E66
:1003E000992799248824002733243092C80008953F
:1003F0006D2DCFEC30E0162F23E07991C198C09A93
:10040000B99AB89A48B357E00000779508F04227A8
:1004100048BB5A95C9F770FF42271A95799148BB96
:1004200091F7582D503041F0779508F0422748BB9E
:1004300000005A95C9F7788100004C7F48BB55E011
:100440005A95F1F7C09AC09AB998B898C09808958B
:100450004091D0004B3443EC09F04BE44093D00082
:10046000089543EC4093D00040E84093CF00F0DF84
:1004700040E04093D1004093D20064E0089548E00A
:10048000A42E40E84093CF0043EC4093D0001A2DB7
:100490006A2DC1EDC895099231966A95D9F762E047
:1004A000610FD2D0639563959394CFEC47D0D62E4D
:1004B0009924D092B1008092B0006D2DFF27EFEC0F
:1004C000C2EB019009926A95E1F7089540E84093E4
:1004D000CC0042ED4093CD000895CF935F938F926F
:1004E000CCEC62E0882486DF8F905F91CF910895F5
:1004F00040E84093C9004AE54093CA0008958F92AE
:10050000C9EC62E0882476DF8F90089540E840933C
:10051000CF004EE14093D00062E00895CF936F93F7
:100520006C0F4FEF47954881242F2795242720955E
:100530002993C617B9F76F91CF91089511277724A2
:100540007A94CF936F93312F48E0340F6A95E9F78F
:1005500026E06F916F936C0F63956395488158E027
:10056000479508F027E02A95A1F4371526E088F48E
:100570003A95732E513011F459E0C3955A9590FA7B
:100580001EF037D01A9502C01BD013956F91CF91F2
:10059000D8CF3A9521F05A9519F7C395DFCF6F91CF
:1005A000CF9190FA3EF0103051F06A95185F38F410
:1005B0006A950895812E185010F06395812E089544
:1005C000452F59E0541B3881331F2FEF220F5A95C6
:1005D000E9F732232095269548814223342B488120
:1005E000441F3993C61301C008953881331F3993CE
:1005F000F9CF452F59E0541B4C2F4395C62F3A9104
:1006000037953883C413FBCF3A9137952FEF5A951E
:1006100011F0220FFCCF3223209548814223342B46
:1006200038830895CF936F93C0E603D06F91CF9135
:1006300008956C0F488138E04795221F3A95E1F7FD
:100640002993C617B9F70895CF936F93CFEC0AD0CB
:100650004095309539934883CA9562E0EADF6F91FF
:10066000CF9108956C0FC3954991433C11F04B34E1
:10067000A9F44FEF3FEF299118E037FB50F95227CB
:10068000441F331F4E7F2695579520F450E8352799
:1006900055E045271A9589F7C61769F70895C89553
:1006A000099231966A95D9F72CC0C895099233FA08
:1006B00036F43196C8950992E89433F802C00024C4
:1006C00009923196625089F71CC0008009923196D8
:1006D0006A95D9F716C0EEBBFFBBE09A0DB209923E
:1006E00031966A95C1F70DC040E84093CF0068E0AD
:1006F000C1ED332009F4D3CF32FCD7CF30FCE5CFA6
:10070000EACF37FC3324A4DEC0ED089506D09394DD
:10071000CFEC14DFD62E9924089533244091620043
:1007200030916300407609F41BC04034B1F0403290
:1007300009F013C0313059F0323051F0333049F004
:10074000393041F03A3039F03B3031F091C090C04F
:100750008FC08EC08DC08CC08BC08AC041E020C0CD
:100760003030E9F03130D1F03330C1F0353079F04C
:10077000363029F1373009F13830A9F0393051F0ED
:100780003A30B9F03B3051F03C30B9F071C0E090F4
:1007900064006EC0409164004093C80069C042E0AC
:1007A000F8E0E8ED52C04091C80041E0F8E0EBEB22
:1007B0004CC0F8E0E2EC41E048C0A8DE089540916A
:1007C0006200413849F030916500313071F03230CB
:1007D00081F03330D9F0089530916500313269F0FD
:1007E000323279F0333289F00895F8E0E4EA42E1F8
:1007F0002CC0F8E0E6EB42E228C0F8E0E8EC49E083
:1008000024C0F8E0EAED4FE620C01FC03CE0332EE4
:10081000309164003030A1F0323051F0333061F06B
:10082000313011F0BBCF24C0F9E0EEE446E80DC052
:10083000F9E0E2E94AE009C0F9E0E8E942E405C08C
:100840003324F9E0EAE444E000C0A0906800A41674
:1008500008F0A42E4A2DBB24477009F0B3944A2D0A
:10086000469546954695B40E43EC4093D0000BC098
:10087000F8DD089502D04BDF08954B2D413011F47F
:10088000F3DD0895BA943A2D385018E018F41A2D73
:10089000BB24B394A32E28DF62E0610FD5DE6395FD
:1008A0006395089512010001000000087707010018
:1008B0000100010200010902220001010280500929
:1008C0000400000103000003092101010001226F5F
:1008D000000705810308000A00000501150009044E
:1008E000A1010502850109BA09BB1581257F75089B
:1008F0009502810205010901A10009360937158118
:10090000257F750895028102093009311600FE26FF
:10091000FF01750A95028102C01601FE09393500F2
:10092000463B011601FE1500250765147504950167
:100930008102850205091901291815002501750193
:100940009518550065008102C00004030900860364
:100950004D696E646175676173204D696C61736187
:1009600075736B61732028632920323030342C205A
:10097000496E672E2049676F72204365736B6F2C39
:1009800020436F7079726967687428632920323058
:1009900030330A034D4A6F7942034D4A6F792C2058
:1009A00041544D6567613820626173656420555319
:0A09B00042204A6F79737469636B8B
:00000001FF
